:020000040000FA
:1000000007309F00A00183168501860183128501B8
:1000100086015B2085175B20851005103F30A50009
:100020004B205B204030A5004B20B830A700A50036
:100030004B20C030A5004B205B20851405100830F4
:10004000A8000230A9004030A6002C18AB0F2D28C4
:10005000AA0A2A08043A0319AA012C144320A5006D
:100060005320A00AA60B2528033085064030A600A1
:10007000A90B2528A70A2708A50085104B20851461
:10008000A80B212842282A08003E8A002B08703E2F
:1000900003188A0A820005112508860085150000CC
:1000A000851100000800051525088600851500004B
:1000B000851100000800FF30642864306428323065
:1000C0006428143064280530A100C730A200013034
:1000D000A300A20B6C28A30B6928A10B6528003490
:1000E0000034003400340034003400340034003470
:1000F0000034003400340034003400340034003460
:10010000003400340034003400340034003400344F
:10011000003400340034003400340034003400343F
:10012000003400340034003400340034003400342F
:10013000003400340034003400340034003400341F
:10014000003400340034003400340034003400340F
:1001500000340034003400340034003400340034FF
:1001600000340034003400340034003400340034EF
:1001700000340034003400340034003400340034DF
:1001800000340034003400340034003400340034CF
:1001900000340034003400340034003400340034BF
:1001A00000340034003400340034003400340034AF
:1001B000003400340034003400340034003400349F
:1001C000003400340034003400340034003400348F
:1001D000003400340034003400340034003400347F
:1001E00000348034E034F034F834FC34FC34FC3433
:1001F000FC34FC34FC34FC34FC34FC34FC34FC347F
:100200007C347C347C347C347C347C347C347C346E
:10021000FC34FC34FC34FC34FC34FC34FC34FC345E
:10022000FC34FC34FC34FC34FC34FC34FC347C34CE
:100230007C347C347C347C347C34FC34FC34FC34BE
:10024000FC34FC34FC34FC34FC34FC347C347C342E
:100250007C347C347C34FC34FC347C347C347C341E
:100260007C347C347C347C347C347C347C347C340E
:100270007C347C347C347C347C347C347C34FC347E
:10028000FC347C347C347C347C347C347C347C346E
:100290007C347C347C347C347C347C347C347C34DE
:1002A0007C34FC34FC34FC347C347C347C347C344E
:1002B0007C347C347C347C347C347C347C347C34BE
:1002C0007C347C347C34FC34FC343C341C341C34AE
:1002D0003C34F834F034E0348034003400340034FA
:1002E0000034FF34FF34FF34FF34FF343F341F3415
:1002F000073407340334013401340034003400344B
:100300000034003400340034F0340034003400345D
:10031000003400340034013401340334033407342E
:100320000F341F347F34FF34FF34FF34FF34003484
:10033000003400340034003400340F340F340F34F0
:100340000F340F340F340F340F340F3400340034B3
:10035000003400340034FF34FF348034003400347F
:10036000003400340434FC34FC34FC34FC34FC34FD
:10037000FC34FC34F83400340034003400340F34DE
:10038000FF34F834003400340034003484348434CE
:1003900084348434843484348434843400340034A5
:1003A000003400341134FF34F834003400340034A5
:1003B00000344434443444344434443444344434C1
:1003C00000340034003400343F34FC3403346334EC
:1003D000633460341F34FF34FF348034003400341D
:1003E0000034FF34FF34FF34FF3400340034003471
:1003F00000340034003400340034333433343334C4
:100400003334333433343334F334333433343334F4
:1004100033343334333400340034003400340034A3
:10042000003400348034FF34FF34FF34FF34E034D0
:100430002034A034A034A034A034BF34BF34FF34FF
:100440003F34FF34FF34FF34FF34FF34F034F034F2
:100450003034B034B034BF34BF34BF34F034F0344F
:100460003034F034F03470349034D034F034D0344C
:10047000D034D0341034D034F034F034F03410347C
:10048000DF34DF34D0343034F034F0343834D8341E
:10049000D834D8343834F834983438347834F8349C
:1004A000F8341834FC34FF34EF340834E834F834CA
:1004B000F834F83408347834B834D834C834F834DC
:1004C0001834E834E834EC341E34FF34FF34FC34A0
:1004D000F034FC34FC34FF34FF34FF348034003417
:1004E0000034FF34FF34FF34FF34FF34FE34F8347B
:1004F000F034F034E034C034C0348034803480349C
:100500008034003400340034033400340034803448
:1005100080348034C034C034E034E034F034F83413
:10052000FC34FE34FF34FF34FF34FF34FF34FF3437
:10053000C034DB34DB34DB34DB34DB34DF34FF3436
:10054000C034DF34DF34DF34DF34DF34DF34FF3412
:10055000C034DD34DD34DD34CD34EF34EF34FF34FA
:10056000E034FD34FA34FB34F734EF34EF34FF3445
:10057000FF34FF34E034FF34FF34FF34FF34E03421
:10058000FE34FC34FA34FB34F734FF34F834F734F7
:10059000F734F734F034FF34FF34F034FF34FE34F2
:1005A000FD34F834F734FF34FF34F834FB34FB34D3
:1005B000FF34FF34F834FF34FE34FD34FB34FF34B1
:1005C000F834FE34FE34FE34F834FF34FF34FF34A4
:1005D000FF34FF34FF34FF34FF34FF34FF34E034A2
:1005E0000034FF34FF34FF34FF34FF34FF34FF3472
:1005F000FF34FF34FF34FF34FF34FF34FF34FF3463
:10060000FF34FF34FF34FF34FF34FF34FF34FF3452
:10061000FF34FF34FF34FF34FF34FF34FF34FF3442
:10062000FF34FF34FF34FF34FF34FF34FF34FF3432
:10063000FF34FF34FF34FF34FF34FF34FF34FF3422
:10064000FF34FF34FF34FF34FF34FF34FF34FF3412
:10065000FF34FF34FF34FF34FF34FF34FF34FF3402
:10066000FF34FF34FF34FF34FF34FF34FF34FF34F2
:10067000FF34FF34FF34FF34FF34FF34FF347F3462
:100680007F347F347F347F347F347F347F347F34D2
:100690007F347F347F347F347F347F343F343F3442
:1006A0003F343F343F343F343F343F343F343F34B2
:1006B0003F343F341F341F341F341F341F341F3462
:1006C0001F341F341F341F341F341F341F341F3492
:1006D0000F340F340F340F340F340F340734033416
:1006E00000340134033407340F340F340F340F3423
:1006F0000F340F340F340F340F340F340F340F34E2
:100700000F340F340F340F340F34073407340734E9
:100710000734073407340734073407340734073401
:100720000734073407340734033403340334033401
:100730000334033403340334033403340334033401
:1007400003340334033401340134013401340134FB
:1007500001340134013401340134013401340134F1
:1007600001340034003400340034003400340034E8
:1007700000340034003400340034003400340034D9
:1007800000340034003400340034003400340034C9
:1007900000340034003400340034003400340034B9
:1007A00000340034003400340034003400340034A9
:1007B0000034003400340034003400340034003499
:1007C0000034003400340034003400340034003489
:1007D0000034003400340034003400340034003479
:1007E0000034003400340034003400340034003469
:1007F0000034003400340034003400340034003459
:100800000034003400340034003400340034003448
:100810000034003400340034003400340034003438
:100820000034003400340034003400340034003428
:100830000034003400340034003400340034003418
:100840000034003400340034003400340034003408
:1008500000340034003400340034003400340034F8
:1008600000340034003400340034003400340034E8
:1008700000340034003400340034003400340034D8
:1008800000340034003400340034003400340034C8
:1008900000340034003400340034003400340034B8
:1008A00000340034003400340034003400340034A8
:1008B0000034003400340034003400340034003498
:1008C0000034003400340034003400340034003488
:1008D0000034003400340034003400340034003478
:02400E00183D5B
:00000001FF
